:100000005EC078C0A7CB76C075C074C073C072C024
:1000100054CB70C06FC06EC08ECB6CC06BC0323022
:10002000313931323033000202020202030303038A
:10003000030304040404040404040405050505057D
:10004000060606060707070808080909090A0A0B31
:100050000B0C0C0D0D0E0F0F1011111213131415A4
:1000600016171818191A1B1C1D1F202122232426BD
:1000700027282A2B2C2E2F3132343537393A3C3E63
:1000800040424446484A4C4E50525456595B5D607B
:100090006265676A6D6F7275787B7D8083868A8DF5
:1000A0009093979A9DA1A4A8ABAFB3B7BABEC2C6AE
:1000B000CACED2D7DBDFE4E8ECF1F6FAFF00112478
:1000C0001FBECFE5D2E0DEBFCDBF10E0A0E6B0E0BE
:1000D000E4E5FCE102C005900D92A637B107D9F71F
:1000E00021E0A6E7B0E001C01D92A331B207E1F71D
:1000F00040DBAECD85CF482FDB0120E030E0C901E9
:1001000063E070E047DDFC01E052FF4F808188230F
:1001100031F02F5F3F4F2031310589F703C0408315
:10012000B283A183089590E822E048EA57E030E0E6
:10013000815070F00FB6F89496BD26BD0FBEFA013F
:100140003197F1F70FB6F89496BD36BD0FBEF0CFDC
:1001500008950F931F93CF93DF938091E00088233E
:1001600009F43FC00091E1001091E200D091E0005D
:10017000C091BD00C150C7FD0DC0EC2FEE0FFF0BAD
:10018000E254FF4F0190F081E02DB8018D2F0995C9
:100190008111F0CF20E030E0F22FE32F2F5F3F4FAF
:1001A000C90163E070E0F6DCDC01A052BF4F4C9166
:1001B0008F2F9E2F63E070E0EDDCFC01E052FF4FDB
:1001C000408311968D919C911297928381832F3059
:1001D000310511F710920D0110920F0110920E01CE
:1001E000BCCFDF91CF911F910F9108959093110192
:1001F00080931001BC01809112017DCF86B383FBF7
:10020000882780F991E089278093BA000895E091CA
:100210006600F09167003196FB70F460F093670020
:10022000E09366008091B6008B5A8093B600E4910B
:100230008091B6008E0F08958093B8008093B70028
:10024000811102C018BC07C08150E82FF0E0E95DC1
:10025000FF4FE491E8BD8091B800863010F492E041
:1002600005C08E3010F491E001C090E080E80FB638
:10027000F89486BD96BD0FBE089581E008958091E3
:10028000A300882369F02091D1003091D200909191
:10029000D000291B821B8093D00082E080937400E1
:1002A0008091A400882319F0835E8093730080916D
:1002B0007300873418F086E480937300089580916A
:1002C000A300811180936800089580939B00B4CFB0
:1002D000CF93C82FCC2351F085E2AEDF82E023DF3D
:1002E00080E0AADF89E11FDFC150F4CFCF910895EC
:1002F000CF93C091B80080E09FDF83E014DF8C2FA4
:10030000CF919ACF0F931F93CF93DF9380919D004E
:100310008093A700809171008093A8008091700065
:100320008093A90080916F008093AA0080916E0055
:100330008093AB0080916D008093AC0080919E0013
:100340008093AD0080916C008093AE0080916A0034
:100350008093AF0080916B008093B0008091690022
:100360008093B100809168008093B2008091A000DA
:100370008093B300809173008093B4008091D0008B
:100380008093B500F89407EA10E0C1E0D1E0F801ED
:1003900061918F01CE014ADC2196C031F1E0DF0787
:1003A000B1F765EA80E091E041DC7894DF91CF918C
:1003B0001F910F91089520919D009091A30080912D
:1003C000A400222381F0911190936F00882321F0E3
:1003D00097E9981B90936E008091A500882361F0A7
:1003E00080936D000895911190937100882321F0FE
:1003F00097E9981B9093700008950F931F93CF93E4
:10040000DF93EC01609171008091700090919D00EC
:10041000992321F060916F0080916E00262F30E0CB
:10042000C217D3070CF440C0282F30E02C173D072B
:10043000E4F180919D00811102C08C2F36C0E091C3
:100440006E0080916F00E81B60916D00F0E070E03D
:1004500061507109CF01CFDB60939C0080916F00E8
:100460006695262F30E010E090916D001917E8F4A2
:1004700040916D0000916F00812F90E0BF018ADBF9
:10048000642F70E061507109A2DB802F860FAE01EE
:10049000481B510957FF03C0519541955109241735
:1004A00035071CF41F5FE0CF862FDF91CF911F919E
:1004B0000F910895FF920F931F93CF93DF938C01B9
:1004C000EB01F42E8091CE009091CF00892B31F07A
:1004D000E091CE00F091CF0089E009951093CF0014
:1004E0000093CE00012B61F0E091CE00F091CF009F
:1004F000BE018F2DDF91CF911F910F91FF90099435
:10050000DF91CF911F910F91FF900895CF93DF93CB
:10051000E091BD00EE2359F0E150E093BD00F0E022
:10052000EE0FFF1FE254FF4FC081D18102C0C0E037
:10053000D0E0E091BD00EE2341F0F0E0EE0FFF1FB0
:10054000E454FF4F8081918102C080E090E04AE056
:1005500060E070E0AFDFCE01DF91CF9108959C01A4
:100560009091BD00983088F4E92FF0E0EE0FFF1F66
:10057000E254FF4F318320839F5F9093BD0048E09A
:10058000C90198DF8091BD0008958FEF08950F9302
:100590001F93CF93DF93EC018B01B8DFB801CE013D
:1005A000DF91CF911F910F91DACFCF93DF93EB01C2
:1005B000883049F480E040DECD2B19F481E080934F
:1005C000B900C0E077C0813021F469317105C8F30A
:1005D000F6CF813B69F481E090E00FDF2DDE809162
:1005E0009D00811102C0689760F361E070E026C051
:1005F000813ED9F3813871F4C0919E00CC2321F063
:100600008C2F90E0FADE22C08091720090E0F5DE3F
:1006100013DE50C0813C71F4C0919E00CC2319F0D0
:100620006C2F70E00BC06091720070E081EE94E07E
:10063000AEDF40C0823B29F466E970E081EE94E0D1
:1006400036C0823CC9F3833919F480E0F5DDB9CFB7
:10065000833C29F460E070E08CEB96E028C0833B9B
:1006600029F460E070E084E999E021C0843C39F429
:1006700082E02EDE60E070E088E993E018C0853CFF
:1006800039F481E025DE60E070E08BE19BE00FC093
:10069000863C39F481E01CDE60E070E082E094E0AA
:1006A00006C08F3C31F460E070E08DE391E06FDFD5
:1006B00088CFC1E08C2FDF91CF910895883049F425
:1006C00010927F0010927E0082E002DE88E1B4DDAD
:1006D00007C0813C39F460E070E085ED92E057DFBF
:1006E00080E00895823C29F460E070E087EC94E0BB
:1006F000F6CF8130D9F480917E0090917F000196F1
:10070000853524E2920728F490937F0080937E0041
:10071000E7CF10927F0010927E008091B800815048
:100720008BDD8091B8008111DBCFD5CF81E00895BA
:100730001F93CF93DF9300D0CDB7DEB7182F80790A
:100740008039C9F480917100898380916F008A8318
:10075000812F8F70823029F490919D0081E089274C
:1007600002C080919D00E1E0F0E0EC0FFD1FE80F7A
:10077000F11D808103C0803819F480E05DDD08C080
:10078000113031F46931710560F01093B90009C07E
:1007900081E0143C39F49CDD60E070E085ED92E08E
:1007A000F6DE80E00F900F90DF91CF911F910895BA
:1007B000843031F58091CE009091CF0029E08439CA
:1007C000920729F469E170E081EE94E017C0815E40
:1007D000944081F48091B800823060F02091B8009C
:1007E0009091B8002695892F86958695820F6DDDAC
:1007F00080E0089560E070E085ED92E0C8DEF8CF1B
:1008000081E00895CF93883061F4C1E0C0937D000A
:10081000C093A00077DDC0937C0085E380937200D5
:1008200036C0813939F480917C00882309F492C064
:1008300086E110C0813841F480917C00882309F45E
:1008400089C08091720006C0823931F481E08093C2
:100850007C0080E0F1DC7EC0813C51F490917C0012
:1008600081E0892780937C00882389F080E00EC096
:10087000813B31F560FD0BC080917C00882349F0FD
:1008800010927C0081E080937D0086E1D5DC80E0E1
:1008900062C09091B8006230710528F4953518F067
:1008A0008FEF80937D0080917D00890F863120F04D
:1008B000863518F085E501C086E180937200E6CFA9
:1008C000813E31F480917D00819580937D00DFCF62
:1008D000863C59F481E0FCDC1092A00013DD60E05E
:1008E00070E085ED92E053DED2CF813081F46E333B
:1008F000710511F480937D0080917C00882339F28A
:100900006F33710520F281E08093B900C0CF85304C
:1009100081F480917C008111BACF8091B80090E081
:10092000861B970B863191050CF0B0CF86E190E0E5
:10093000ADCF843079F49091B8008091B80096954D
:1009400086958695890F863108F0A0CF81E0809347
:100950007C009DCF81E0CF910895813C29F460E037
:1009600070E085ED92E006C0823C31F460E070E01A
:100970008CEB96E00CDE07C0843C39F460E070E05C
:1009800084EB96E0ECDD80E0089581E00895813C01
:1009900029F460E070E085ED92E006C0823C31F41D
:1009A00060E070E08DEA94E0F2DD07C0843C39F449
:1009B00060E070E088EB96E0D2DD80E0089581E0B1
:1009C0000895CF93DF939B0140917100C091700017
:1009D00090919D00992339F040916F00C0916E0075
:1009E000D0919C0001C0D1E0982F9D7F9830B9F440
:1009F0001092A2008A3019F42091720030E0842F06
:100A000090E08217930730F4D0E02C173D0710F4E4
:100A100020937200C901F1DC58DC81E081C0813C87
:100A200031F460E070E085ED92E0B1DD67C1823CB9
:100A300049F48091B800863910F486E995C0809118
:100A4000720092C0833C81F490919D0081E09111ED
:100A500080E080939D0056DC4BDC8091B80090E0F4
:100A6000CCDC8093720080C0843C31F460E070E0A4
:100A70008EEA96E074DD42C1813B09F04CC0809162
:100A80009D00882339F0C90168E170E0A0D8892B66
:100A900009F034C12115310571F48091B8008C172B
:100AA00010F08FEF05C08091B8004817C8F081E0C2
:100AB0008093650015C0273381E0380788F0809166
:100AC000B8008C1770F72D36324050F08091B80086
:100AD000481730F00DDC60E070E088E993E057DD06
:100AE0002091B800809165006D2F70E0082E000CF9
:100AF000990B50D8820F911D80DCD82F8093720003
:100B00008091B800D81729F0D13411F0CD1301C06D
:100B1000EFDB8D2F29C0813E31F4809165008195F6
:100B200080936500EBC0823B09F581E0809365000E
:100B300080919D00882339F0C90168E170E047D8B1
:100B4000892B09F0DBC08091B80090E08D1B9109E2
:100B500054DCC82F809372008091B800C81719F038
:100B6000C13409F4C5DB8C2FB0DBC8C0853C29F447
:100B70008091B80080939E0007C0853B41F4232BF1
:100B800009F0BEC010929E00BDDBB2DBB9C081305F
:100B900009F06BC02E33310511F48093650080910C
:100BA000B7002091B80090E0821B91094091850028
:100BB000509186004F5F5F4F5093860040938500B1
:100BC000009709F49BC097FF07C02091B8002A3610
:100BD00030F020E430E005C020E032E002C020E048
:100BE00031E03695279597FD019695958795009765
:100BF000C1F72417350708F081C08091B7009091A4
:100C0000B800891720F48091B800815007C09091F6
:100C1000B800981718F48091B8008F5F2FEF280F55
:100C2000E22FF0E0E95DFF4F94913091B800231777
:100C300028F428B5211102C09F3F59F028B5291783
:100C400018F498B59F5F05C028B5921718F498B5A9
:100C5000915098BD98B5E4919E1302C08093B8005E
:100C6000109286001092850049C08530B1F48091C1
:100C7000B800823408F442C08091B80090E0821B32
:100C8000930B8134910534F087399105A8F186E9F9
:100C900090E032C081E490E02FC08630C1F49091A2
:100CA000B80080919B00981748F59091B800290FE3
:100CB000311D90E08217930734F02134310524F47C
:100CC00021E430E001C09C012093B70017C08730B9
:100CD000B9F49091B7008091B800891720F4809101
:100CE000B8008F5F09C09091B7008091B800981745
:100CF00028F48091B80081508093B70080E001C053
:100D000081E0DF91CF910895883029F410927B0023
:100D100080E092DA21C0813089F480917B008617CF
:100D200040F4682F70E06F5F7F4F8EEC96E017DC29
:100D300013C0FA010995E6DAE9DB0EC08A3061F4E6
:100D400080917B0090919F00E82FF0E0ED55FF4FE0
:100D500090838F5F80937B0080E0089560919D0079
:100D60006E5F4BED51E0D0CF4FE351E062E0CCCF6E
:100D70004FE551E061E0C8CF813C29F460E070E0CC
:100D800085ED92E006C0823C39F460E070E08EE5CB
:100D900093E0FDDB80E0089581E00895CF93DF9339
:100DA000883059F410927A0060937900109278009C
:100DB000109277001092760085C0813009F068C0EB
:100DC00090917800892F8D7F81F420917600309169
:100DD00077002F31310538F42F5F3F4F3093770084
:100DE0002093760072C09F5F25C0913051F58091AD
:100DF00079008823F1F0C0917600D09177009E01B0
:100E00002F7133272A30310511F485E204C02431D3
:100E1000310519F480E010DA06C02F31310519F4DC
:100E20008150809379002196D0937700C09376000B
:100E300049C092E09093780010927700109276006B
:100E400044C09330E9F4C0917600D09177002196A8
:100E5000D0937700C0937600CE01837099270097D6
:100E600011F489E103C0029711F482E1E5D9CB3B8B
:100E7000D10540F180E0E0D984E08093780022C081
:100E8000943001F580917A0080939F003FDB1AC077
:100E90008138D1F41092120181E08093A6008091F4
:100EA0007800833079F480917A008F5F80937A00A4
:100EB00010927700109276008BE4BED984E033D98B
:100EC00080E0BAD980E001C081E0DF91CF91089540
:100ED0000F931F93CF938091DF00882309F41FC1E4
:100EE0001092DF0024B195B13091B600229526957D
:100EF00026952370892F90E0880F991F880F991FDE
:100F0000820F911D830F8093B6008091D4008823B7
:100F100009F405C11092D4008091DD0081113CC01C
:100F200080917400882349F06091D9007091DA00B3
:100F30007093D6006093D50004C06091D500709185
:100F4000D600605F7F4FA6E076956795AA95E1F79A
:100F500080E098E53CD66B5F7F4F76956795609310
:100F6000D30080919A00882311F0815009C08091AC
:100F7000D3008D3138F460E070E084E0BCD885E0C7
:100F800080939A008091B9008111C0C08FEA87B91F
:100F900081E08093DD00B5C0813009F0B7C0809159
:100FA0007400811143C08091D7009091D800409681
:100FB0009C0145E0369527954A95E1F7A091D00030
:100FC000A901569547950A2E000CBB0BCD01835104
:100FD0009140840F951F9093D2008093D10080910F
:100FE0008900E82FF0E0EE0FFF1FE657FF4F40812A
:100FF0005181B901641B750B318320838F5F87702A
:1010000080938900CB01880F991F880F991F409109
:10101000730050E04D5E5E4F4A1B5B0B440F551F43
:10102000841B950B820F931F23E01CC08091DB0073
:101030009091DC009093D8008093D700409635E0E3
:10104000969587953A95E1F7EAE8F0E081939193D8
:1010500020E0EA39F207D1F7A6CF009709F0019610
:10106000215029F018161906C4F70197F9CF181660
:101070001906E4F477FD39C02091880012160CF1AE
:10108000880F991FBC016350710977FF02C06F5F21
:101090007F4F759567951616170614F061E070E09E
:1010A00088E1861B8093880085E026C08C3F2FEF67
:1010B0009207DCF477FF19C02091880027FF05C054
:1010C0002450281B2093880018C024EE281B20934E
:1010D00088002091D3002F3180F06CEF7FEF681BE8
:1010E000790B7595679586E007C08091D3008E31A6
:1010F00020F060E070E087E0FED78CE287B91092C4
:10110000DD001092DE0086B1886486B9809174009B
:10111000882329F08091740081508093740080911D
:10112000BC00882309F476C01092BC0080911001A5
:10113000909111019C012F5F3F4F88279078822B5F
:10114000932B9093110180931001C091BA0056D84F
:10115000C817F1F01092B9002091120110921101FC
:1011600010921001922F882331F090692F702F3048
:1011700041F09F5F06C09F7E25FD02C0906801C0C0
:10118000906C909312018093BA0080E090E02ED88A
:101190000091100110911101C09112018C2F807FDC
:1011A000803B19F460E070E001C0B80181E0A3D792
:1011B000C4FF0EC0C5FF02C0C80108C00831110538
:1011C000C8F0C062C093120180E090E00FD812C056
:1011D000CC2381F0C5FD09C00231110558F0C0646F
:1011E000C093120180E090E001D81092120181E0DA
:1011F0008093A60080918700811106C086B1886423
:1012000086B981E08093D400809187008F5F8F71D1
:1012100080938700CF911F910F910895AF92BF9255
:10122000CF92DF92EF92FF920F931F93CF93DF93B2
:10123000E090CE00F090CF00EC0110E800E088E0F4
:10124000C82E87E0D82E92ECA92EBB24B394209709
:1012500041F18091B800863040F482E00FB6F894F6
:1012600016BD86BD0FBEC50106C00FB6F89416BDEB
:1012700006BD0FBEC6010197F1F70FB6F89416BD73
:1012800006BD0FBE25DE8091A60081110CC0209105
:10129000CE003091CF002197E216F30629F459D7FA
:1012A000D6CF81E001C080E0DF91CF911F910F91F7
:1012B000FF90EF90DF90CF90BF90AF900895CF93C5
:1012C000C82F882381F08EE1B7D786EA90E0A6DFA9
:1012D00080E0B2D78AEF90E0A1DFC150A1F78AE9A0
:1012E00092E0CF919BCF8EE1A7D789E190E096DF86
:1012F00080E0A2D78AEF90E091DFF1CFCF93DF9328
:1013000064E659D4282F892F6AE055D4EC012223B2
:1013100041F0822FD4DF8C2FD2DF8D2FDF91CF9140
:10132000CECFC111F8CFF9CFCF92DF92EF92FF92DB
:101330000F931F93CF93DF93EB01E0916C0091E04B
:101340009093A200E33009F0E5C0883029F41092B0
:10135000840090936300E0C0823C19F410928400F2
:10136000E9C0813BC9F420916200CD2B51F42E36A7
:1013700020F08FEF8093630004C0223010F490932C
:10138000630080916300820F11F481E048C18F36C1
:1013900008F445C18EE643C1813E31F4809163007B
:1013A000819580936300FCC0823B59F49093630065
:1013B00080916200823008F4FBC08150809362000B
:1013C000F7C0833C79F480918400843E08F019C111
:1013D000855E809384008091B800805E2DD782E086
:1013E000A2D60FC1813009F003C16E33710511F42B
:1013F0008093630020918400FE01FF70213069F426
:101400008091620090E04996BF0134E0769567953F
:101410003A95E1F7BFD3C92E01C0C12CEF3FFF4081
:1014200061F4222351F0215020938400211105C042
:1014300060E070E085ED92E0AAD8D09083008D2D19
:10144000880FD7FC809590E067E070E0A3D3492F28
:10145000E09082008E2D880FE7FC8095009161005E
:10146000602F70E090E096D3F09081003F2D330F15
:10147000F7FC309510916000809162008C19840F08
:10148000282F290F612F70E0832F90E083D3822FC4
:10149000890F87FD80E0D0D6C0FD05C0B8D6817029
:1014A000D80ED092830080918000E80EE0928200F6
:1014B000AED665E280D3F90EF0928100A8D68F7384
:1014C00029F4A5D66DE077D390938000002331F006
:1014D0009ED68F7319F401500093610098D6811144
:1014E00007C095D66BE067D390936100109282009D
:1014F000133030F08CD68F7119F4115010936000B6
:1015000086D68F7709F07FC082D666E054D3909359
:10151000600079C0883021F481E08093640081C04C
:10152000813C31F460E070E085ED92E030D879C024
:10153000823C49F48E2F90E0019665E070E05BD329
:1015400080936C005AC0813B49F5E23088F460FD1D
:1015500068C0F0E0E659FF4F808190916400891BDC
:10156000883020F08F3F99F58EEF31C088E02FC092
:10157000E43009F056C09091690080916400890FB1
:101580008093690080916900823010F482E02AC063
:1015900080916900893740F188E724C0813E31F4A9
:1015A0008091640081958093640027C0823B19F587
:1015B00081E080936400E23060F4C0FD32C0F0E06E
:1015C000E659FF4F80818F3F61F180818F5F80837B
:1015D00028C0E43031F580916900833028F0809193
:1015E00069008150809369008091690025D619C0F7
:1015F000813C09F497CF823E11F484D612C0813029
:1016000011F081E00FC0CE33D10519F481E0809351
:1016100064008091B600C80FC093B60002C08093EA
:10162000620080E0DF91CF911F910F91FF90EF90CA
:10163000DF90CF9008950F931F93CF93DF93D82F10
:101640008B01883031F48091A200813011F488E060
:101650006BDE8D2F8079803959F481E08093A10071
:10166000C091A200C1110AC080917200E5D51FC0CF
:10167000803831F41092A10080E0DED5C0E017C0C0
:10168000D130A1F4C091A100CC2351F08091A200EF
:101690008130A1F7B801DF91CF911F910F9144CE16
:1016A0000733114058F3D093B90001C0C1E08C2F2B
:1016B000DF91CF911F910F9108951F920F920FB656
:1016C0000F9211242F933F938F939F93AF93BF93C8
:1016D000EF93FF938091DE008823E9F0E091DD0035
:1016E00024B135B1F0E0EE0FFF1FDF01A752BF4F6D
:1016F0002D933C93EB52FF4F80819181821793078A
:1017000008F401962817390708F40197918380831C
:1017100081E08093DF0081E08093DE00FF91EF9114
:10172000BF91AF919F918F913F912F910F900FBEDD
:101730000F901F9018951F920F920FB60F921124C1
:101740008F9381E08093BC008F910F900FBE0F901C
:101750001F9018951F920F920FB60F9211248F931E
:1017600081E08093BB008F910F900FBE0F901F9070
:101770001895F89484B7877F84BF0FB6F894A8951E
:1017800081B5886181BD11BC0FBEB99A81E083BF6C
:1017900081EA8ABD88E088BB85BB8BB780628BBF3E
:1017A000A89581B5886181BD80E481BD8CE287B94F
:1017B0001092DD001092DE0086B1886486B987EE53
:1017C00086B9789481E0AFD460E070E088ED93E072
:1017D000C6D682E131D583E0A6D480E02DD50ED5E2
:1017E000811108C0F89480E091E018D2853A69F13F
:1017F000789476C0C0E08C2F1FD583E190E00EDD99
:101800008C2F869519D583E190E008DDF7D48823E5
:1018100099F0CF5FC03479F785E18093A3001092EF
:10182000A4002DD56FD5C6E98C2F06D584E090E0B5
:10183000F5DCC150C9F7D6CFCC23A1F28C2FFCD454
:101840008DE090E0EBDCC150F7CF07EA10E0C1E09B
:10185000D1E0CE01E3D1F80181938F012196C0310F
:10186000F1E0DF07B1F778948091A70080939D00A5
:101870008091A800809371008091A90080937000EE
:101880008091AA0080936F008091AB0080936E00DE
:101890008091AC0080936D008091AD0080939E009C
:1018A0008091AE0080936C008091AF0080936A00BD
:1018B0008091B00080936B008091B10080936900AB
:1018C0008091B200809368008091B3008093A00063
:1018D0008091B400809373008091B5008093D00014
:1018E0008091A000882329F065E370E082E094E015
:1018F00004C061E070E085ED92E031D622242394AB
:1019000042E0342E5CE2452E67EE562E70E4972EB0
:10191000E7E08E2ECC24C394D12CA5E07A2EBDE036
:101920006B2ECCEFAC2EC3E0BC2E13D48091B9004B
:101930008823A9F180E080D4A89584B7877F84BFED
:1019400081B5886181BD11BC379858D48111FDCF14
:10195000109212012092A6008BB780628BBF10926A
:10196000B90085B7877E806185BF85B7806285BFF6
:10197000889585B78F7D85BF309274008BB78F7D3A
:101980008BBF47B81092DD001092DE0086B18864EC
:1019900086B956B8A89581B5886181BD91BC98DAA1
:1019A0008091CE009091CF0021E08D339207A1F479
:1019B000CEE1D0E0FE018491805381DC8CE291E0A5
:1019C0002DDC2196F0E0C632DF07A1F760E070E081
:1019D00085ED92E0DCD5DBC029E08439920779F00F
:1019E0003BE08B31930709F09FC08091A2008130CA
:1019F00009F0C3C08091A100882309F4BEC0C09142
:101A00006C00C23001F120F0C43009F476C0BFC0D0
:101A1000EC2FF0E0E659FF4FD08186E90DD4C111DB
:101A200009C0DA3220F4C5010197F1F707C081E05F
:101A300090E003C08D2F869590E0F0DB80E0FCD332
:101A40008D2F90E098C0E3D38F73E82EF12CDFD375
:101A5000682DB1D0E60102C0CC0FDD1F9A95E2F7E8
:101A6000D6D3672DA8D0F60102C0EE0FFF1F9A95BE
:101A7000E2F7CE0FDF1FCBD390E0BE01BCD0C80F82
:101A8000D91FC739D10514F0C6E9D0E08C2FD4D3C3
:101A9000C701C4DB8E0133E0159507953A95E1F750
:101AA000011101C001E010E0C701B8DBC01BD10B80
:101AB000D7FF02C0C0E0D0E08C2FBED3A8D3837084
:101AC00031F4C701ABDBCE0195958795B5D3C23014
:101AD000D10554F79CD3662D6ED0E60102C0CC0F21
:101AE000DD1F9A95E2F793D390E0BE0170D0C80F46
:101AF000D91F80E0A1D3CE013EC0C0916900CC0FB8
:101B0000C73908F0C6E9D4E08C2F96D385E090E081
:101B100085DB8091690090D381E490E07FDBD15038
:101B200099F780ED92E027C0F6E08C3B9F0721F407
:101B30008091D300E3DB2BC024E0873C920789F43B
:101B40008091720079D384E690E068DB80E074D302
:101B50008091680090E068EE73E01CD08456910993
:101B60000AC08D5A944049F48091D1009091D200DE
:101B7000C5DB88EE93E052DB0AC085B7877E85BF60
:101B800085B7806285BF889585B78F7D85BF1092A8
:101B9000A600CBCE0024552704C0080E591F880F7D
:101BA000991F009729F076956795B8F37105B9F7F5
:101BB000802D952F0895991B79E004C0991F9617E1
:101BC00008F0961B881F7A95C9F780950895AA1B7F
:101BD000BB1B51E107C0AA1FBB1FA617B70710F018
:101BE000A61BB70B881F991F5A95A9F7809590954A
:101BF000BC01CD01089597FB072E16F4009406D082
:101C000077FD08D0E4DF07FC05D03EF49095819580
:101C10009F4F0895709561957F4F0895E199FECF8C
:101C20009FBB8EBBE09A99278DB30895262FE1992B
:101C3000FECF9FBB8EBBE09A01970DB2021639F022
:101C40001CBA2DBB0FB6F894E29AE19A0FBE089524
:041C5000F894FFCF36
:101C5400060B180101010004024129430307780A15
:061C64007801412D020091
:00000001FF
